:100000000429AD0001300428A6002E082C02031D8F
:100010000B282D082B02043003180130031902307D
:100020002605031D0130FF288030A100FE30A420EA
:100030000130A4207530AC003030CF28A101A117C9
:10004000B400FE30A4203408A428A501AF00B001FC
:10005000A01125080319A0150530A4002730AE0013
:1000600010303E200330AE00E8303E20AE01643058
:100070003E20AE010A303E202F084528AD00300852
:10008000AC002F08AB00E3202B08AB00A40303193E
:10009000A011250803194F282402031856282B08FD
:1000A000031DA011A0195628303EA4280800B20054
:1000B000061186118316061186110F3086058312EC
:1000C0003208A01881283E30AC008030CF20333079
:1000D000B10095201330AC008830CF2095206430DB
:1000E000CE2095206430CE202230B10095202830DB
:1000F00080200C30802006308020A0143208812817
:100100002014B100201C8F288611033C031C942866
:1001100094200530AC00DC30CF20031408002014FC
:10012000FE3C0319A2288615201C201006150F304E
:1001300086053108F03986040611B10E201895287D
:100140003230CE203208FF28A11B572883169B008F
:1001500083161C141A089B0AFF2883169A001C1584
:1001600055309D00AA309D009C149C18B5281C1188
:100170009B0AFF2883178001840AFF3E031DBB28CA
:10018000FF28AE01AD00FF30AD07031CAE07031C16
:10019000FF280330AC00DF30CF20C328AC01E83E9D
:1001A000AB00AC09FC30031CD828AB070318D528DA
:1001B000AB070000AC0FD5282B18DE28AB1CE228BB
:1001C0000000E2280800B001AF011030B1002C0D92
:1001D000AF0DB00D2D08AF022E08031C2E0FB0027C
:1001E0000318F9282D08AF072E0803182E0FB007A3
:1001F0000310AB0DAC0DB10BE7282B08FF288313C0
:100200008312031300000800A00107309F0083162B
:10021000FF308500FC30860081178312850186013E
:10022000203084006030BB20A03084005030BB20E0
:10023000203084003030BA200130AE00F430C220CB
:100240008614851A6729BC14142054305720453071
:10025000572053305720543057204D3057204F30BF
:10026000572044305720453057202C3057207930C4
:1002700057206F305720753057202030572063307B
:100280005720613057206E3057208030A100C03099
:100290001E2072305720653057206C305720653053
:1002A0005720613057207330572065305720203059
:1002B0005720623057207530572074305720572010
:1002C0006F3057206E305720851A67296429142013
:1002D00043305720613057206C305720572065300D
:1002E0005720723057202030572049305720443053
:1002F000572020305720553057204B305720203082
:100300005720563057202D3057203130572080301D
:10031000A100C0301E2077305720572057202E30A4
:100320005720703057206930572063305720623093
:100330005720613057207330572069305720633081
:1003400057202E3057206E3057206C305720073002
:10035000AE00D030C2200130A620A7002708031D20
:10036000B329BC146D2D0301A620D6000130A620B0
:10037000DA000330D9000230A620A700A70803192D
:10038000C229061402305A020318C829CA21C929F1
:10039000E121072C14204E3057206F305720203099
:1003A00057206E305720753057206D3057206230FF
:1003B0005720653057207230572073305720302235
:1003C00008001420503057207230572065305720D5
:1003D00073305720653057206E30572074305720C7
:1003E0003A305720203057208030A100A501FF303F
:1003F0005A07AF00FF300318013EB000282020301C
:1004000057206E3057207230572003305A02031C99
:100410000D2A273057207330572006182F2A803096
:10042000A100C0301E204E3057206F3057202030A2
:1004300057206E30572065305720773057202030B6
:1004400057206E305720753057206D30572062305E
:1004500057206530572072305720733057200800DE
:10046000BC1C3E2A8030A100CC301E2054305720C6
:100470004530572053305720543057200800D801BA
:100480008030A100C0301E204D30572065305720ED
:100490006D3057206F3057207230572079305720F9
:1004A0002030572066305720753057206C30572049
:1004B0005720051E5C2A592A851E732ADC0A04303F
:1004C000C120FB305C02031C6F2A023086068316B3
:1004D0008610831286180614861C0610DC01051E81
:1004E000722A4A2B5C2A0614072C02305802031881
:1004F0007A2A072C0614023083169B0001308312DF
:10050000AD200330D700DB01FF305A07A700FF30D2
:100510000318013EA8002808031D922A27085B0241
:100520000318CB2A3C14DB0ADC01DC0A5C083D3EE4
:1005300084000008A7005708A620A9000F3029054D
:10054000AA01A9002A08031DA92A290827020319BC
:10055000AA2A3C10D70A5708A620A700F030270582
:10056000A801A7002808AC002708AB00AE010301D2
:100570000120BB0003305C020301031801303B057E
:100580000319952A58085C020319C72A3C103C1C21
:10059000CA2ACB2A842A3C18182B560A83169B0099
:1005A000F0308312AD200130DC00B801F030B7002C
:1005B0005608A620A7002708B705B801BA010F30D2
:1005C000B9005C083D3E84000008A9002908B9056F
:1005D000BA0137083904DD00560883169B008312E0
:1005E0005D08AD20DC0A7B3056020318F92AD60AD2
:1005F000FA2A3F2A5C0858020318D52ADA0A560854
:1006000083169B0083125A0EB700B800F030B7056E
:100610000F30B8053708AD203808AD2083169B0190
:1006200083125608AD205A08AD200130AD20432B6F
:100630000330D7005708A620DC00D70AA8015C0EBB
:100640000F39A7002808031D1A2B27085B02031D7A
:100650001A2B5708A620A700F0302704DC00570803
:1006600083169B0083125C08AD200130DC00013052
:1006700086068316061064308312C120DC0A2930F6
:100680005C02031C372B051E462B432B3230C12046
:100690003C10072C0130C120030105180130B801BE
:1006A000B700BA010230B9003908851C0301B9004E
:1006B0003A08851C0301BA003908B7073A0803183D
:1006C000013EB807BA010430B9003908051D03011D
:1006D000B9003A08051D0301BA003908B7073A08FE
:1006E0000318013EB807BA010830B9003908851D62
:1006F0000301B9003A08851D0301BA00370839071C
:10070000D5000B30550203190130031D0301BB0056
:100710000301BC1801303B05BB005508031901302B
:10072000031D03013B040319A42B14204E30572052
:10073000723057203A305720302283301E20A101DA
:1007400086143C150330D9003C1DDA2B55080319DB
:10075000AD2B0B305502031DAE2BD92B55080319B9
:10076000CA2B0B3055020318CA2B0A305502031D41
:10077000BA2BD5018030A10055082520D80A580889
:100780003D3E8400550880000F305802031CC92BE1
:10079000752AD92B0C305502031DD22BBC1CD12B32
:1007A000752AD92B0F305502031DD82B752AD92B4A
:1007B000072CDB2B072C3A30D1009830D0000301F6
:1007C000051A0130BB005108AC005008AB00AE0167
:1007D000030101203B050319F42B6430CE20D00324
:1007E000500A0319D103DF2B3A30D1009830D000E2
:1007F000051A062C6430CE20D003500A0319D10309
:1008000051085004031D052C752AF82B4A2B75300E
:10081000CF003030CE003C11D801DC015C083D3EF9
:10082000840000308000DC0A10305C02031C0E2CB7
:10083000851A1B2C2B2C051E1E2C4A2B4F084E04F0
:10084000031D242C86102A2C0130C120CE034E0A11
:100850000319CF03182C86147530CF003030CE002A
:1008600004305602031C0F2DD301D201D20A031902
:10087000D30A0A30C120061C3F2CD301D201851EA9
:10088000422C472C5208C83A5304031D362C5308F7
:10089000031D4E2CC8305202031C4F2C102D59083A
:1008A000A620D40014208030A100C0301E204E307D
:1008B0005720723057203A305720A501F0305405A8
:1008C000B801B7003708AF003808B0000430AB00FB
:1008D0000310B00CAF0CAB0B682C28202F30572026
:1008E000A501FF305A07AF00FF300318013EB000EA
:1008F0002820590ADC005C08A620A7001030270237
:10090000031C962C203057202A3057204E30572079
:100910002A3057205C08A620A7000F302705DD00ED
:100920005C0883169B0083125D08AD203022803066
:100930001E20A1018030A100A5010F305405B00197
:10094000AF002820D90A5908A620D400103054023C
:10095000031C9A2CF0305405B801B7003708A700E3
:100960003808A8000430AB000310A80CA70CAB0B90
:10097000B42C2808031DC22C27085A02031DC22CC0
:100980000330D900061CE32C0330D7005708A620FB
:10099000A700F0302705A801A7002708F03A28048F
:1009A000031DD32CD82CD70A7B305702031DC62C2D
:1009B0007B305702031DDD2C0610023083169B008E
:1009C00003018312AD20851AE62CE32C0A30C120E6
:1009D000D301D201D20A0319D30A0130C1204F0832
:1009E0004E04031DF52C8610F92CCE034E0A031974
:1009F000CF03061CFD2CD301D201851A002D2B2C10
:100A0000051E032D4A2B53083A3A98300319520613
:100A1000031DEA2C06180D2DE1210330D900072C07
:100A200014204530572072305720613057207330E2
:100A3000572065305720203057206E3057207530B2
:100A400057206D3057206230572065305720723064
:100A50005720733057203F3057208030A100C030DE
:100A60001E204230572055305720543057205720F1
:100A70004F3057204E305720203057203D305720E0
:100A800020305720433057206F3057206E3057208A
:100A90006630572069305720723057206D3057200C
:100AA0003022851A542D512D0A30C120C830DC0067
:100AB0000301851A0130BB0001305C0203010318F9
:100AC00001303B050319682D1430C120DC03582D7B
:100AD0005C08031D6D2DE121072C14204E3057209A
:100AE000753057206D3057206230572065305720C1
:100AF00072305720733057202030572061305720F4
:100B000072305720653057208030A100C0301E2041
:100B1000653057207230572061305720733057208E
:100B20006530572064305720213057203022033061
:100B300083169B0010308312AD200430D600560877
:100B400083169B0003018312AD20D60A7C30560227
:100B5000031C9F2D0130DC00013086068316061031
:100B6000C8308312C120DC0A0B305C02031CAC2DA0
:100B7000CA210330D6000130DA000330D900061054
:100B800083169B0183125608AD205A08AD2003013D
:0E0B9000AD20851ACC2DC92D0A30C120072CAE
:02400E00103F61
:084200000300000000001000A3
:00000001FF
